:1000000037C1000052C1000050C100004EC10000C5
:100010004CC100004AC1000048C1000046C10000B8
:1000200044C1000042C100000C94630D3EC10000B9
:100030003CC100003AC1000038C1000036C10000D8
:1000400034C1000032C1000030C100002EC10000E8
:100050002CC100002AC1000028C1000026C10000F8
:1000600024C1000022C1000020C100001EC1000008
:100070001CC100001AC1000018C1000016C1000018
:1000800014C1000012C1000010C100000EC1000028
:100090000CC100000AC1000008C1000006C1000038
:1000A00004C1000002C1000000C1000005010904F4
:1000B000A101A1027501950D15002501350045012D
:1000C00005091901290D81029503810105017504B6
:1000D00095012507463B0165140939814265009564
:1000E000018103A10075029504250245020930092A
:1000F00031093209358102C0C07508950826FF0014
:1001000046FF000600FF09200921092209230924CE
:1001100009250926092709280929092A092B950CE7
:1001200081020A2126B102C005010904A101A10230
:10013000850175089501150026FF0081037501955D
:100140001315002501350045010509190129138101
:10015000027501950D0600FF8103150026FF0005BD
:10016000010901A10075089504350046FF0009301A
:100170000931093209358102C00501750895270941
:1001800001810275089530090191027508953009C1
:1001900001B102C0A1028502750895300901B102C2
:1001A000C0A10285EE750895300901B102C0A10217
:1001B00085EF750895300901B102C0C01201100128
:1001C0000000004010008200010001020001120145
:1001D0001001000000404C0568020100010200010E
:1001E00009022200010100C0FA0904000001030015
:1001F0000000092111010001227C00070581034054
:10020000000109022900010100C0FA0904000002EE
:1002100003000000092111010001229400070502DA
:100220000340000107058103400001040309042283
:100230000341006B006900680061006200610072A8
:10024000006100730068006F0070002E006A00708B
:100250000000001A03500053003300360030002B1A
:10026000002000760031002E003000300000000039
:1002700011241FBECFEFDAE0DEBFCDBF12E0A0E059
:10028000B1E0E8E0F3E202C005900D92AC30B107B6
:10029000D9F712E0ACE0B2E001C01D92AD33B10776
:1002A000E1F70E94870B0C948211AACE2FB1209502
:1002B000237379B1A3B1A095A077FC0161E06083BD
:1002C000118215821286138614861586128E138E5D
:1002D000148E10A211A212A213A252E054A34FEF47
:1002E00045A387E786A367A390E890A7558F8FEE75
:1002F000868F84E1878F128213821686108A118A74
:100300001786148A128A158A138A118E108E178AFC
:10031000168A1482968397839087918780911F0213
:1003200030E0882341F121FF03C0109220021BC05E
:1003300024FF03C06093200216C025FF03C0509322
:10034000200211C020FF0FC080910B01882359F0BB
:1003500080911E02882319F460931E0202C010923D
:100360001E0210920B01A4FF12C110921F0281E025
:1003700080930B01089521FF22C0809120028823E1
:10038000B1F480E182834687C9018072907024FFB6
:1003900007C0892B09F083C080E98283418B7FC02D
:1003A000892B09F47CC080E38283478778C0813041
:1003B00011F4178227C0823011F4118635C020FF56
:1003C0003FC0809120028823C9F44281842F806439
:1003D00082835FEF508BC9018072907024FF07C049
:1003E000892B09F05CC0406C4283518B58C0892B2B
:1003F00009F455C040664283578751C0813081F46B
:100400004FEF4783C9018072907024FF04C0892B8D
:1004100009F045C027C0892B09F441C046833FC07D
:10042000823071F44FEF4187C9018072907024FFD0
:1004300003C0892BA1F51CC0892B89F140872FC0EF
:1004400024FF18C080912002882341F425FD27C095
:100450008281806882838FEF818B21C0813021F47B
:1004600025FD1DC016821BC0823021F425FD17C05A
:10047000108615C025FF13C080912002882331F417
:100480008281806282838FEF878709C0813019F46F
:100490008FEF868304C0823011F48FEF8087972F0F
:1004A0009095292F30E090FF05C083818068838379
:1004B0008FEF818FB9016270707021FF05C0838159
:1004C000806183838FEF868B22FF05C083818860E4
:1004D00083838FEF858B23FF05C0838184608383B3
:1004E0008FEF848B24FF05C08381806483838FEF2B
:1004F000808F25FF05C08381806283838FEF878B88
:1005000026FF05C08381826083838FEF838B97FFF3
:1005100005C08381816083838FEF828B4A2F50E0F7
:100520009A0120713070A4FF03C0828188608283A9
:1005300045FF1FC0828181608283672B29F181E0A2
:1005400080931F0221C0209121023091220281E07C
:100550002C32380738F080911E02882319F481E08C
:1005600084830BC02F5F3F4F3093220220932102E0
:1005700004C0109222021092210246FF08C081E0BE
:10058000848380931E020895232B99F3DCCF089572
:100590002FB12095237369B153B150955077FC0169
:1005A0004FEF4283148215821682178285E583837A
:1005B0001082118210861186128613861486158683
:1005C0001686178680911F0230E0882349F121FFAB
:1005D00003C0109220021CC024FF02C081E003C0AF
:1005E00025FF04C082E08093200212C020FF10C0CB
:1005F00080910B01882361F080911E02882321F4F1
:1006000081E080931E0202C010921E0210920B0124
:1006100054FF2BC110921F0281E080930B010895BB
:1006200021FF3CC0809120028823B1F4C90180726F
:10063000907024FF07C0892B61F487E08283468392
:10064000458398C0892B29F081E0828346834483C7
:1006500091C0128246838EC0813079F4C9018072C4
:10066000907024FF04C0892B31F480E582C0892B6F
:1006700011F082E57EC081E57CC0823079F4C90149
:100680008072907024FF04C0892B31F485E071C022
:10069000892B11F085E26DC085E16BC020FF3EC063
:1006A000809120028823C1F4C9018072907024FFD8
:1006B00007C0892B61F485E082838FEF878339C07F
:1006C000892B29F083E082838FEF878349C084E000
:1006D00082838FEF87834EC0813079F4C9018072A5
:1006E000907024FF04C0892B31F488E542C0892B27
:1006F00011F08AE53EC089E53CC0823079F4C90139
:100700008072907024FF04C0892B31F485E831C0D9
:10071000892B11F085EB2DC085E92BC024FF17C074
:1007200080912002882339F425FD24C086E082834D
:100730008FEF85831FC0813021F425FD1BC084E528
:1007400018C0823021F425FD15C085E412C025FFB4
:1007500011C080912002882329F482E082838FEFE8
:10076000848308C0813011F486E503C0823011F41F
:1007700085E68383962F9095292F30E090FF05C062
:100780008081816080838FEF8387B9016270707090
:1007900021FF05C08081886080838FEF808722FFE2
:1007A00005C08081806280838FEF858723FF05C02D
:1007B0008081806180838FEF848724FF05C08081E2
:1007C000826080838FEF828725FF05C080818460EF
:1007D00080838FEF818726FF05C0808180688083BA
:1007E0008FEF878797FF05C08081806480838FEFBC
:1007F0008687452F50E09A012071307044FF03C076
:1008000081818260818345FF20C0818181608183F5
:10081000672B41F181E080931F0224C020912102C7
:100820003091220281E02C32380740F080911E0284
:10083000882321F48181806181830BC02F5F3F4F2A
:10084000309322022093210204C0109222021092BF
:10085000210246FF0AC081818061818381E080930B
:100860001E020895232B89F3D9CF0895239A1CBC27
:100870008CB580648CBD8CB580628CBD8CB5886075
:100880008CBD8CB584608CBD0895982F2F9A8DB542
:1008900081118EB59EBD90E025E008C0822F8A951B
:1008A000F1F79F5F993C11F48AEA08950DB407FEB1
:1008B000F5CF61112F988EB508953F924F925F92B8
:1008C0006F927F928F929F92AF92BF92CF92DF9260
:1008D000EF92FF920F931F93C82E81E090E020E8E3
:1008E0000FB6F89420936100809361000FBE84B12D
:1008F000807784B985B1876085B9B8DF279A2F9A48
:1009000000E0FF24FA94F0E8DF2EE5E3AE2E73E773
:10091000B72E69E7962E51E4852E4CEF742E3FE7F3
:10092000632E2FEE522E9FEC492E8FE6382E2F9AF3
:10093000FEBC1899FCCF9FB190959373F9B1F095D7
:10094000E3B1E095E077F0920101F0920201D092DC
:100950000301D0920401D0920501D09206011092B9
:100960000C0210920D0210920E0210920F021092C1
:1009700010021092110210921202109213021092A1
:100980001402109215021092160210921702809112
:100990001F02492F50E0882349F191FF03C01092B4
:1009A00020021CC094FF02C081E003C095FF04C078
:1009B00082E08093200212C090FF10C080910B0152
:1009C000882361F080911E02882321F481E08093C6
:1009D0001E0202C010921E0210920B01E4FF54C1CD
:1009E00010921F0281E080930B014EC191FF23C042
:1009F000809120028823A9F450920101F0920E0206
:100A00009A012072307094FF06C0232B09F089C030
:100A10003092010160C0232B09F483C04092010190
:100A20002AC0813019F4109204012CC0823019F4CC
:100A30001092060138C040FF41C0809120028823F7
:100A4000E9F490910101892F8F7B80930101F0924D
:100A50000F029A012072307044FF07C0232B09F067
:100A600060C09F739093010136C0232B09F459C0D5
:100A70009F7990930101F0920C0253C0813079F478
:100A8000F09204019A012072307044FF04C0232BBD
:100A900009F047C027C0232B09F443C03BC0823074
:100AA00069F4F09206019A012072307044FF03C08D
:100AB000232BB9F51EC0232BA1F131C044FF1CC06C
:100AC00080912002882351F445FD2BC080910101C3
:100AD0008F7780930101F0920D0223C0813029F4B9
:100AE00045FD1FC0109203011CC0823029F445FD52
:100AF00018C01092050115C045FF13C08091200257
:100B0000882331F4809101018F7D80930101B3CF5F
:100B1000813019F4F092030104C0823011F4F09294
:100B200005012F2F30E0F0FF04C060920201F09227
:100B30001102B9016270707021FF07C0809102013B
:100B40008F7E80930201F092100222FF07C08091F5
:100B50000201877F80930201F092150223FF07C0F4
:100B6000809102018B7F80930201F092140224FF96
:100B700007C0809102018F7B80930201F0921202E4
:100B800025FF07C0809102018F7D80930201F092C2
:100B9000130226FF07C0809102018D7F809302011E
:100BA000F0921702F7FF07C0809102018E7F8093B9
:100BB0000201F09216024E2F50E09A01207130701F
:100BC000E4FF05C080910101877F8093010145FF0B
:100BD0004CC0809101018E7F80930101672B09F445
:100BE00045C281E080931F0241C2209121023091D1
:100BF00022022F30310590F180911E02882371F579
:100C000083E0C81659F5809100018823A9F1F0927C
:100C10000201D0920301D0920401D0920501D0923A
:100C2000060110920C0210920D0210920E02109208
:100C30000F021092100210921102109212021092E2
:100C400013021092140210921502109216021092C2
:100C5000170270920101109200010EC02F5F3F4FEA
:100C6000309322022093210207C010922202109298
:100C7000210281E08093000146FF06C083E0C81690
:100C800019F481E080931E028FEF61E0FEDDE82E13
:100C900081E0E81609F0E2C180911802882309F486
:100CA00018C183EF61E0F1DD182F8AE561E0EDDD29
:100CB000163409F48FC0173490F4133409F43FC08C
:100CC000143430F41034D9F0113409F0C7C120C005
:100CD000143409F44DC0153409F0C0C168C01C3487
:100CE00009F4A5C01D3420F4173409F0B7C194C02D
:100CF0001D3409F4BDC01F3409F0B0C1D6C080E076
:100D000061E0C3DD082F80E061E0BFDD82E0D7C095
:100D100080911902813041F48FEF61E0B6DD8FEFF1
:100D200061E0B3DD83E0CBC080E061E0AEDD80E078
:100D300061E0ABDD80E061E0A8DD80E090C080E0B4
:100D400061E0A3DD082F80E061E09FDD80E061E0ED
:100D50009CDD80E061E099DD80E061E096DD80E08F
:100D600060E093DD002309F079C11092180276C18A
:100D700080E061E08ADD082F80E061E086DD80E0D0
:100D800061E083DD80E061E080DD80E061E07DDDC9
:100D900080E060E07ADD013029F4B0920701009331
:100DA00019025CC1809207011092190257C183E0B9
:100DB00061E06BDD082F82E061E067DD8091190260
:100DC000813009F080E061E060DD82E061E05DDDBE
:100DD00081E048C080E061E058DD082F882359F4A5
:100DE00080E061E052DD81E061E04FDD82E061E0C2
:100DF0004CDD80E00DC0813009F030C180E061E061
:100E000044DD81E061E041DD81E061E03EDD81E0E3
:100E100061E03BDD8FE029C080E061E036DD80E00D
:100E200061E033DD82E061E030DD80E0CFCF80E063
:100E300061E02BDD082F882341F480E061E025DDAF
:100E400080E061E022DD84E00AC0813009F006C163
:100E500080E061E01ADD80E061E017DD87E061E0BD
:100E600014DD80E061E011DD80E060E00EDDF6C0C1
:100E70008091080161E009DD8093080180910901FA
:100E800061E003DD809309018FEF61E0FEDC8FEF0D
:100E900061E0FBDC8FEF61E0F8DC8FEF60E0F5DC18
:100EA000B0920701E0921902D9C09092070180E048
:100EB00061E0EBDC082F80E061E0E7DC80E061E0EE
:100EC000E4DC80E061E0E1DC80E061E0DEDC8AE53A
:100ED000CCCF8091070161E0D8DC182F8AE561E072
:100EE000D4DC80910701813449F48091010161E0F3
:100EF000CCDC082F8091020160E0C7DC8091070103
:100F0000833759F58091010161E0BFDC082F8A3AEF
:100F100009F4A4C08091020161E0B7DC8A3A09F4C7
:100F20009DC08091050161E0B0DC8A3A09F496C069
:100F30008091060161E0A9DC8A3A09F48FC08091B2
:100F4000030161E0A2DC8A3A09F488C080910401BF
:100F500060E09BDC8A3A09F481C0809107018937FF
:100F600009F076C08091010161E08FDC082F8A3A98
:100F700009F474C08091020161E087DC8A3A09F4C7
:100F80006DC08091050161E080DC8A3A09F466C099
:100F90008091060161E079DC8A3A09F45FC08091B2
:100FA000030161E072DC8A3A09F458C080910401BF
:100FB00061E06BDC8A3A09F451C080910C0261E077
:100FC00064DC8A3A09F44AC080910D0261E05DDC7C
:100FD0008A3A09F443C080910E0261E056DC8A3AF5
:100FE00009F43CC080910F0261E04FDC8A3AB1F114
:100FF0008091100261E049DC8A3A81F1809113020C
:1010000061E043DC8A3A51F18091120261E03DDCFB
:101010008A3A21F18091110261E037DC8A3AF1F0DD
:101020008091140261E031DC8A3AC1F080911502AE
:1010300061E02BDC8A3A91F08091160261E025DCB8
:101040008A3A61F08091170260E01FDC8A3A31F041
:10105000133421F4013011F4009318022F9A03C0C5
:101060008A2D8A95F1F7189962CCFACF232B09F4CF
:10107000FCCDBBCD84B7877F84BF88E10FB6F894E1
:1010800080936000109260000FBE81E090E020E845
:101090000FB6F89420936100809361000FBE84B175
:1010A000807784B985B1866085B985B1867085B948
:1010B00088B18F7388B981B38F7381BB87B18F7308
:1010C00087B980B38F7380BB729A76986A9A6E9A4A
:1010D00080B38C7C80BB81B3836381BB8AB11AB837
:1010E0008BB18FEF8BB984B18F7884B985B180676C
:1010F00085B9089508950895AF92BF92DF92EF9257
:10110000FF920F931F93DF93CF93CDB7DEB7C054F9
:10111000D0400FB6F894DEBF0FBECDBFADB6BEB6A1
:10112000D0901C02DD2009F0CBC0809136028530C2
:1011300009F484C0863020F4813009F02BC207C046
:10114000863009F449C0893009F024C287C08091F3
:101150003502813A09F01EC2809138028E010F5F7C
:101160001F4F833071F588E0F80111928A95E9F7F5
:101170008091E800877F8093E80060913B02709146
:101180003C02C801EBD68091E8008B778093E800A1
:1011900080911D02882309F0FDC1F8948091E00040
:1011A00081608093E00080E49CE90197F1F781E0A1
:1011B00080931C028091E0008E7F8093E000789401
:1011C000E9C1C801E5D98091E800877F8093E800F4
:1011D000C80160E170E0A1C080913502803809F05B
:1011E000D9C18091370290913802292F80509140C7
:1011F00099F480913B0290913C028830910511F066
:10120000429751F4809123028F5F80932302809153
:1012100024028F5F80932402223049F480913B02A4
:1012200090913C028055914009F0B4C111C0233027
:1012300009F0B0C181E080932502ACC180913502F4
:10124000882309F0A7C180912402813009F0A2C14E
:10125000809123028F5F809323029CC1809135028D
:10126000882309F097C180912502882329F4809171
:1012700023028F5F8093230280912302853008F43C
:1012800089C1F8948091E00081608093E000A7D349
:1012900080E49CE90197F1F7109223021092240256
:1012A00072986E988CE291E020E931E0F901319773
:1012B000F1F70197D9F783E080930A01FEDA6AC15A
:1012C00031E0D31609F066C120913602213021F0B9
:1012D000293009F05FC195C080913502813A09F04B
:1012E00059C18091370290913802E3E081309E0726
:1012F000D9F4DE011196ECECF1E080E401900D925E
:101300008150E1F78091E800877F8093E800609149
:101310003B0270913C02CE01019620D68091E800FC
:101320008B778093E80036C1F3E0823F9F0751F44A
:10133000DE011196ECE8F1E080E401900D9281501D
:10134000E1F7E0CF33E0853F9307C9F4DE01119662
:10135000ECE4F1E080E401900D928150E1F780919E
:101360002F02813079F6DE011196E6E2F2E088E0A4
:1013700001900D928150E1F710922F02C3CFE3E06C
:101380008F3E9E0769F4DE011196ECE0F1E080E407
:1013900001900D928150E1F780912E028887B2CFA3
:1013A0008E010F5F1F4F885F9340F9F480E4F801CE
:1013B00011928A95E9F792E09A8383E08D838E8378
:1013C0002F8380EB88879A8B85E78B8B9C8B86E7B6
:1013D0008D8B99AB8091E800877F8093E8006091C6
:1013E0003B0270913C02C80198CFC8010E9456018F
:1013F0008091E800877F8093E800C80161E370E096
:101400008CCF80913502813209F0C4C080913702BF
:1014100090913802F3E08F3E9F0721F5FDB6EEB6BE
:1014200060913B0270913C022DB73EB7261B370BF3
:101430000FB6F8943EBF0FBE2DBF0DB71EB70F5F9E
:101440001F4F8091E800877F8093E800C801ECD5AA
:101450008091E8008E778093E800F8018681809380
:101460002E022EC0F3E0853F9F0769F5FDB6EEB66C
:1014700060913B0270913C022DB73EB7261B370BA3
:101480000FB6F8943EBF0FBE2DBF0DB71EB70F5F4E
:101490001F4F8091E800877F8093E800C801C4D582
:1014A0008091E8008E778093E80026E232E0409158
:1014B0003B0250913C02C901B8011BD7D0922F02C8
:1014C0002F2D3E2D62C032E081309307E9F5FDB645
:1014D000EEB660913B0270913C028DB79EB7861BC1
:1014E000970B0FB6F8949EBF0FBE8DBF0DB71EB7FA
:1014F0000F5F1F4F8091E800877F8093E800C8014D
:1015000093D58091E8008E778093E8003E983F98CD
:1015100086988798F8018185823011F43E9A0BC035
:10152000843011F43F9A07C0883011F4869A03C0C2
:10153000803109F4879A8F2D9E2D9C010FB6F89467
:101540003EBF0FBE2DBF26C0845F934019F50EB776
:1015500060913B0270913C022DB73EB7261B370BC2
:101560000FB6F8943EBF0FBE2DBF8091E800877F75
:101570008093E8008DB79EB7019656D58091E8001C
:101580008E778093E8002A2D302F0FB6F8943EBF57
:101590000FBE2DBF0FB6F894BEBE0FBEADBEC05C71
:1015A000DF4F0FB6F894DEBF0FBECDBFCF91DF91F6
:1015B0001F910F91FF90EF90DF90BF90AF90089533
:1015C00080911C02813031F461EC42E380D182E0F1
:1015D00060EC02C081E061EC42E379C10F931F939C
:1015E000DF93CF93CDB7DEB760970FB6F894DEBF29
:1015F0000FBECDBF809134028430E9F481E0809346
:10160000E9008091E80080FF16C08E010F5F1F4F38
:10161000C8010E94C802C80160E170E040E050E0EB
:1016200003D68091E8008E778093E80080E1F8018E
:1016300011928A95E9F760960FB6F894DEBF0FBE57
:10164000CDBFCF91DF911F910F9108950F931F93FD
:10165000DF93CF93CDB7DEB7E1970FB6F894DEBF37
:101660000FBECDBF80913402843079F582E0809343
:10167000E9008091E80082FF10C08091E80085FFBA
:1016800007C0CE01019661E370E040E050E07AD5FA
:101690008091E8008B778093E80081E08093E900F7
:1016A0008091E80080FF11C08E010F5F1F4FC801BD
:1016B0000E945601C80161E370E040E050E0B4D5FB
:1016C0008091E8008E778093E800E1960FB6F89459
:1016D000DEBF0FBECDBFCF91DF911F910F91089557
:1016E00080E090E020E80FB6F894209361008093AA
:1016F00061000FBED0D1789480911C02813011F42A
:10170000A5DF03C0882309F469DFE0D5F5CFB2DC9B
:1017100080E49CE90197F1F789B1809580FF09C0C9
:1017200010921C0281E080931D0240E020E030E036
:1017300023C081FF04C081E080931C02F4CF82FFAC
:1017400012C072986E988CE291E020E931E0F901C4
:101750003197F1F70197D9F781E080931D0283E07B
:1017600080930A0107C084FFE0CF81E080931D02CF
:1017700080910A01A2D8D9CF199B06C083B190E00D
:1017800083709070892B31F480910A0196D840E0E3
:1017900020E030E0642F6F5F81E0641708F080E0A4
:1017A000582F520F81E0521708F080E0830F91E02C
:1017B000831708F090E0462F252F382F992351F4F6
:1017C000853040F48430C1F6543920F45339A1F601
:1017D000603E90F285DF80E090E00895DA0120918C
:1017E0001C02222391F59330A1F0943030F4913013
:1017F00051F0923009F063C009C09132F1F0923299
:1018000009F05DC01DC0ECEBF1E032C0E0EEF1E0AC
:1018100034C0813051F0813020F0823009F04FC067
:1018200008C0EBE2F2E084913DC0EFE2F2E0849187
:1018300039C0E3E5F2E0849135C0E2EFF1E037C072
:10184000ECEAF0E02CE730E03EC0213009F037C090
:101850009330B1F0943028F4913041F0923079F522
:101860000AC0913211F1923251F524C0EEECF1E050
:1018700022E130E028C0E2E0F2E029E230E023C0DB
:10188000813049F0813018F08230C9F408C0EBE2B1
:10189000F2E0849107C0EFE2F2E0849103C0E3E557
:1018A000F2E08491282F30E00EC0E4E1F2E029E07C
:1018B00030E009C0E8E2F1E024E930E004C0E0E013
:1018C000F0E020E030E0ED93FC93C9010895382F5B
:1018D000282F2CC02093E900231721F4762F942F72
:1018E00050E006C07091EC009091ED005091F00036
:1018F00091FF1BC08091EB008E7F8093EB00809165
:10190000ED0082708093ED008091EB008160809308
:10191000EB007093EC009093ED005093F0008091F9
:10192000EE0087FD02C080E008952F5F273090F21F
:101930003093E90081E008958091350288239CF47A
:1019400004C0809134028823B9F08091E80082FFBE
:10195000F8CF8091E8008B778093E800089580911C
:101960003402882349F08091E80080FFF8CF80910D
:10197000E8008E778093E80008954091E40050914C
:10198000E50024E68091EC0080FF05C08091E8002E
:1019900080FF05C022C08091E80082FD1EC08091BA
:1019A0003402882311F482E00895853011F483E035
:1019B00008958091EB0085FF02C081E00895809139
:1019C000E4009091E50084179507E1F2222311F4D9
:1019D00084E008952150AC01D5CF80E0089566D011
:1019E0006DD0E0EEF0E0808181608083A8EDB0E012
:1019F0008C918F778C9319BCE7EDF0E080818E7F1E
:101A000080838C918F7E8C93109233020895EF9295
:101A1000FF920F931F934AD051D008ED10E0F801C8
:101A20008081982F9F7790838068808380818F7DCD
:101A3000808319BC1092340210923202109231024B
:101A40001092300280EEE82EF12CF70180818B7F1E
:101A50008083F80180818160808380E060E042E3E0
:101A600036DFE1EEF0E080818E7F8083E2EEF0E011
:101A7000808181608083808188608083F70180819C
:101A80008E7F8083F8018081806180831F910F9118
:101A9000FF90EF900895E7EDF0E080818160808312
:101AA0008AE482BF81E080933302B1CFE8EDF0E0B9
:101AB00080818E7F80831092E20008951092DA0078
:101AC0001092E10008951F920F920FB60F92112409
:101AD0002F933F934F935F936F937F938F939F9336
:101AE000AF93BF93EF93FF938091E10082FF0AC011
:101AF0008091E20082FF06C08091E1008B7F80939D
:101B0000E1002BD28091DA0080FF1EC08091D800C6
:101B100080FF1AC08091DA008E7F8093DA00809176
:101B2000D90080FF0DC080E189BD89B5826089BD83
:101B300009B400FEFDCF81E080933402DBDA04C0FB
:101B400019BC10923402D7DA8091E10080FF18C0EE
:101B50008091E20080FF14C08091E2008E7F80932C
:101B6000E2008091E20080618093E2008091D800E1
:101B700080628093D80019BC85E080933402EDD157
:101B80008091E10084FF2EC08091E20084FF2AC092
:101B900080E189BD89B5826089BD09B400FEFDCFB1
:101BA0008091D8008F7D8093D8008091E1008F7E56
:101BB0008093E1008091E2008F7E8093E20080912B
:101BC000E20081608093E20080913202882331F448
:101BD0008091E30087FD02C081E001C084E0809332
:101BE0003402BBD18091E10083FF22C08091E200EA
:101BF00083FF1EC08091E100877F8093E10082E037
:101C000080933402109232028091E1008E7F8093A3
:101C1000E1008091E2008E7F8093E2008091E200FB
:101C200080618093E20080E060E042E350DE95D185
:101C3000FF91EF91BF91AF919F918F917F916F91A4
:101C40005F914F913F912F910F900FBE0F901F907A
:101C500018950F931F93DF93CF93CDB7DEB7AC9753
:101C60000FB6F894DEBF0FBECDBF8091F100809318
:101C700035028091F100809336028091F1009091BD
:101C8000F100E7E3F2E0809337029093380280910D
:101C9000F1009091F1008093390293838091F100DB
:101CA0009091F10080933B02958326DA8091E800C1
:101CB00083FF3AC18091350230913602353009F404
:101CC00087C0363040F43130C9F1313070F03330F4
:101CD00009F02AC133C0383009F4F8C0393009F4AA
:101CE00007C1363009F020C199C0803821F0823810
:101CF00009F01AC108C09091300280913102882306
:101D000099F0926011C08091390287708093E90048
:101D10008091EB0090E025E0969587952A95E1F774
:101D2000982F91701092E9008091E800877F80934E
:101D3000E8009093F1001092F100D3C0882319F0CD
:101D4000823009F0F1C090E08F719070009721F01F
:101D5000029709F0E9C00CC080913702813009F088
:101D6000E3C010923102333069F5809331022AC00A
:101D700080913702882331F520913902277009F4C8
:101D8000D3C02093E9008091EB0080FF1BC033306B
:101D900021F48091EB00806213C08091EB008061A0
:101DA0008093EB0081E090E002C0880F991F2A9594
:101DB000E2F78093EA001092EA008091EB008860DD
:101DC0008093EB001092E9008091E800877F8CC03F
:101DD000882309F0A9C0109137021F770FB7F89434
:101DE0008091E800877F8093E800A6DD8091E8007D
:101DF00080FFFCCF8091E3008078812B8093E3000B
:101E00008091E30080688093E300112311F482E065
:101E100001C083E0809334020FBF86C080588230B7
:101E200008F082C0809137029091380223E08C3D07
:101E3000920709F033C083E08C838AE28B837FB7FB
:101E4000F894DE0115966EE040E050E011E2E62FD6
:101E5000F0E010935700849140FF03C082958F708B
:101E60006F5F8F70282F30E08A3018F0C901C79655
:101E700002C0C901C0968D939D934F5F5F4F44315F
:101E8000510529F77FBF8091E800877F8093E800A4
:101E9000CE0103966AE270E061D012C0609139020F
:101EA000AE014F5F5F4F9ADCBC01009709F43CC064
:101EB0008091E800877F8093E80089819A81FAD039
:101EC0008091E8008B778093E8002EC0803861F520
:101ED0008091E800877F8093E800809132028093B0
:101EE000F1008091E8008E778093E80025DD1CC02A
:101EF0008823D1F4909137029230B0F48091E800B9
:101F0000877F8093E8009093320216DD8091320241
:101F1000882331F48091E30087FD02C081E001C095
:101F200084E0809334024CDB8091E80083FF0AC098
:101F30008091EB0080628093EB008091E800877FC6
:101F40008093E800AC960FB6F894DEBF0FBECDBF0D
:101F5000CF91DF911F910F91089508959C014091B9
:101F60003B0250913C024617570718F4F90190E0E4
:101F700045C06115710511F0AB01F8CF8091E80003
:101F80008E778093E80040E050E0F0CF80913402FB
:101F9000882309F445C0853009F444C08091E800E5
:101FA00083FF02C081E008958091E80082FD32C085
:101FB0008091E80080FF22C08091F3009091F200B0
:101FC000782F60E0292F30E0262B372B07C0819136
:101FD0008093F100415050402F5F3F4F4115510514
:101FE00019F02034310598F390E02034310509F4DC
:101FF00091E08091E8008E778093E80041155105CB
:1020000029F6992319F606C080913402882341F0FD
:10201000853041F08091E80082FFF6CF80E008959E
:1020200082E0089583E008959C016115710529F40B
:102030008091E8008B778093E800F90127C08091B8
:102040003402882399F1853099F18091E80083FF6B
:1020500002C081E008958091E80082FFF0CF06C0C1
:102060008091F10081936150704059F02091F3000C
:102070008091F200322F20E090E0822B932B892B6D
:1020800079F78091E8008B778093E80061157105FE
:10209000B1F606C080913402882341F0853041F0CA
:1020A0008091E80080FFF6CF80E0089582E00895F7
:1020B00083E008959C0140913B0250913C024617F9
:1020C000570718F4F90190E046C06115710511F049
:1020D000AB01F8CF8091E8008E778093E80040E074
:1020E00050E0F0CF80913402882309F447C0853056
:1020F00009F446C08091E80083FF02C081E00895A2
:102100008091E80082FD34C08091E80080FF23C008
:102110008091F3009091F200782F60E0292F30E059
:10212000262B372B08C084918093F10031964150C3
:1021300050402F5F3F4F4115510519F020343105B4
:1021400090F390E02034310509F491E08091E800AB
:102150008E778093E8004115510521F6992309F007
:10216000C1CF06C080913402882341F0853041F010
:102170008091E80082FFF6CF80E0089582E0089524
:1021800083E00895BF92CF92DF92EF92FF920F9378
:102190001F93CF93DF93182F092F7B016A01EDDB8B
:1021A000B82E8823B1F5812F902F9C01E901C1142D
:1021B000D10439F0F60180819181E81AF90AC80F3B
:1021C000D91F00E010E022C08091E80085FD16C014
:1021D0008091E8008B778093E800C114D10449F026
:1021E000F60180819181800F911F9183808385E02A
:1021F00011C06CD0C2DB882349F00CC08091F10083
:1022000089930894E108F1080F5F1F4FE114F1046E
:10221000D9F68B2DDF91CF911F910F91FF90EF9009
:10222000DF90CF90BF900895BF92CF92DF92EF9250
:10223000FF920F931F93CF93DF93182F092F7B01EA
:102240006A019BDBB82E8823B1F5812F902F9C016A
:10225000E901C114D10439F0F60180819181E81AB5
:10226000F90AC80FD91F00E010E022C08091E800F1
:1022700085FD16C08091E8008E778093E800C11438
:10228000D10449F0F60180819181800F911F9183E3
:10229000808385E011C01AD070DB882349F00CC020
:1022A00089918093F1000894E108F1080F5F1F4FB6
:1022B000E114F104D9F68B2DDF91CF911F910F918D
:1022C000FF90EF90DF90CF90BF9008951F93809183
:1022D0003402882361F01091E9001092E9008091A6
:1022E000E80083FF01C0B5DC17701093E9001F916F
:1022F0000895FB01DC0102C001900D924150504055
:08230000D8F70895F894FFCF0F
:1023080001FFFF8080808041FFFF040100EF020091
:10231800030301A000000000000000000002030108
:102328008F020801910201018B01F3007C0000007B
:102338000000000000000000000000000200000093
:102348000000000000000000000000000100001371
:10235800A9DEE77498490003408818018A00000044
:102368000000040002020202000000040404040049
:10237800000106000000000000000000000000004E
:10238800000000000000000000000000F2FFFF0055
:102398000019C16198490003408818018A000000AB
:1023A8000000040002020202000000040404040009
:1023B800000106000000000000000000000000000E
:1023C8000000000000000000000000000001020002
:1023D8000308010217171717090A00000000000078
:1023E80000000400020202020000000404040400C9
:1023F80000010600000000000000000000000000CE
:0C240800000000000000000000000000C8
:00000001FF
